:020000020000FC
:1000000012C01895189518951895189537C034C0D2
:1000100037C018951895189518951895189518952E
:100020001895189518950FE50DBF04E00EBF0FEF5A
:1000300004BB00E001BB0FEF05BB82E19AE79BBD6B
:100040008ABD89E09DE399BD88BD09B7086109BFF4
:100050000CE00EBD7894879906C088B599B50196D5
:1000600099BD88BD0FD0869906C088B599B501970E
:1000700099BD88BD07D0EFCFA8981895A89A189574
:0C008000A89A18950FEF0A95F1F7089563
:00000001FF
